:100000000EC01DC01CC01BC01AC04CC018C017C0F9
:1000100016C015C014C013C013C011C010C01124E5
:100020001FBECFE5D2E0DEBFCDBF20E0A0E6B0E04E
:1000300001C01D92A236B207E1F746D05AC0E0CF08
:100040001F920F920FB60F9211242F933F938F930D
:100050009F9380916000909161009C012150310933
:100060003093610020936000892B99F4C39B07C0F3
:1000700083E190E0909361008093600006C080EF80
:1000800090E0909361008093600098B388E18927A5
:1000900088BB9F918F913F912F910F900FBE0F9032
:1000A0001F9018951F920F920FB60F9211248F93E5
:1000B0009F9398B385E0892788BB9F918F910F907C
:1000C0000FBE0F901F9018958DE187BB91E098BBF4
:1000D00080E481BD23E130E0309361002093600033
:1000E00088B3886188BB93BF89B7826089BF7894E1
:0600F000FFCFF894FFCFE2
:00000001FF
